S021000064656D6F70726F675F6F6C696D65785F73746D3332653430372E73726563A1
S3150800C00018080020BDF3000805F4000809F4000824
S3150800C0100DF4000811F4000815F4000800000000EB
S3150800C02000000000000000000000000019F40008ED
S3150800C0301DF400080000000021F4000893D9000848
S3150800C04025F4000829F400082DF4000831F4000846
S3150800C05035F4000839F400083DF4000841F40008F6
S3150800C06045F4000849F400084DF4000851F40008A6
S3150800C07055F4000859F400085DF4000861F4000856
S3150800C08065F4000869F400086DF4000871F4000806
S3150800C09075F4000879F400087DF4000881F40008B6
S3150800C0A085F4000889F400088DF4000891F4000866
S3150800C0B095F4000899F400089DF40008A1F4000816
S3150800C0C0A5F40008A9F40008ADF40008B1F40008C6
S3150800C0D0B5F40008B9F40008BDF40008C1F4000876
S3150800C0E0C5F40008C9F40008CDF40008D1F4000826
S3150800C0F0D5F40008D9F40008DDF40008E1F40008D6
S3150800C100E5F40008E9F40008EDF40008F1F4000885
S3150800C110F5F40008F9F40008FDF4000801F5000834
S3150800C12005F5000809F500080DF5000811F50008E1
S3150800C13015F5000819F500081DF5000821F5000891
S3150800C14025F5000829F500082DF5000831F5000841
S3150800C15035F5000839F500083DF5000841F50008F1
S3150800C16045F5000849F500084DF5000851F50008A1
S3150800C17055F5000859F500085DF5000861F5000851
S3150800C18065F5000869F50008EE11AA55C2788A18FF
S3150800C190DFF84432DA7083780A0092B2120AD218AB
S3150800C1A0DFF834329A704278DFF82C325A70027807
S3150800C1B0DFF824321A70DFF8202293780A0092B248
S3150800C1C0120A92B2934212DADFF80C225278521C03
S3150800C1D0DFF804325A70DFF800225278002A06D1B6
S3150800C1E0DFF8F4211278521CDFF8EC311A70DFF808
S3150800C1F0E821D27889B201F0FF039A421CDADFF807
S3150800C200D8219278521CDFF8D0319A70DFF8C8210D
S3150800C2109278002A10D1DFF8C0215278521CDFF834
S3150800C220B8315A70DFF8B0215278002A04D16A4A28
S3150800C2301278521C684B1A707047F0B40D0092B20F
S3150800C24001EB0206761E3400A5420ED22E7836027F
S3150800C2506F78F6193300181806001F00B6B2BFB279
S3150800C260BE4200D2401CAD1CEEE7A5420AD12E788C
S3150800C27036023300181806001F00B6B2BFB2BE4217
S3150800C28000D2401C80B2F0BC704710B51422534946
S3150800C2900020FFF7D2FF0400A4B2002C02D14FF60B
S3150800C2A0FF7003E0200080B201F060F880B210BD94
S3150800C2B070B504004A48007C00024949497C401888
S3150800C2C01438050055FA84F006000822454930005E
S3150800C2D080B2FFF7B2FF06002A0092B24249300048
S3150800C2E080B2FFF7AAFF0600B6B2002E02D14FF6BB
S3150800C2F0FF7003E0300080B201F038F880B270BDFC
S3150800C30080B50620FFF7D4FF02BD00203749087024
S3150800C3103648007800280BD100203549334A127870
S3150800C32021F8120031480078401C30490870EFE7C0
S3150800C33000202E4908702D48007800280DD10020CD
S3150800C3402C492A4A12781E235A431144487627480C
S3150800C3500078401C25490870EDE74FF480602649AF
S3150800C360088070470021214A117020490978002960
S3150800C37012D11F491D4A127831F81210002905D129
S3150800C3801B491A4A127821F8120005E0174909785C
S3150800C390491C164A1170E8E7704710B504002100D9
S3150800C3A089B2164800680830FFF7F0FE0A48007898
S3150800C3B0124909680872084840781049096848729D
S3150800C3C0054880780D49096888720348C0780B4982
S3150800C3D00968C87210BD0000C81C00202608002085
S3150800C3E018080020320800203A080020E01C002027
S3150800C3F0D41C0020801B0020D81C0020C01C002054
S3150800C40038B50400DFF8D00C0568DFF8D00CDFF883
S3150800C410EC1C0860DFF8E40C0068DFF8E41C086030
S3150800C420E4B2032C11D1687E10F00F0003280AD15C
S3150800C430288A002807D10820DFF8A41C087000F015
S3150800C440F9FF00F00FBE00F086BFE4B2022C40F000
S3150800C450A780DFF8A00DC078401CDFF8981DC870CB
S3150800C460DFF8900DC07800281ED1DFF8880D807897
S3150800C470401CDFF8801D8870DFF8780D807800286A
S3150800C48012D1DFF8700D4078401CDFF8681D48703F
S3150800C490DFF8600D4078002806D1DFF8580D0078DF
S3150800C4A0401CDFF8501D08700020DFF84C1D08807E
S3150800C4B00020DFF8481D0880687E072802D0687EBD
S3150800C4C0052808D1A87E401CA876A87E782865D1BC
S3150800C4D00020687662E0687E00285FD0288A0028F7
S3150800C4E04FD0A87E411EA976C0B2002856D1E87E54
S3150800C4F0082808D0687E022802D0687E012811D153
S3150800C500E87E05280ED1002068768020DFF8D01B4B
S3150800C510087000F08FFF1420DFF8E41C81F82F0064
S3150800C52000F07EBEE87E052801DB042000E0E87EF8
S3150800C530032111FA00F0A876E87E401CE876687EAA
S3150800C54010F00F00C0B201280AD0022809D003282B
S3150800C5500DD0042813D0062811D008280FD01DE0C6
S3150800C5600DE30020DFF8981C81F82F000CE3042067
S3150800C570DFF86C1B087000F05DFF00F0B8BD00F036
S3150800C58014BD687E10F00F00032807D10820DFF8D5
S3150800C590501B087000F04EFF00F064BD00F0DBBED3
S3150800C5A0DFF85C0C807B452840F0D586DFF8480C20
S3150800C5B00088DFF84C1C097C0902DFF8442C527C01
S3150800C5C08918884211DBDFF8380C007C0002DFF896
S3150800C5D0301C497C4018DFF8201C0880DFF8200C46
S3150800C5E0007D3F21084207D101E000F0B4BEDFF824
S3150800C5F0100C407D002801D000F0ADBEDFF8640DB8
S3150800C6000088DFF8641D0988884207D1DFF8540DD1
S3150800C6104088DFF8541D4988884211D0DFF8E00BBE
S3150800C620C08BDFF8401D0988884207D1DFF8D00B98
S3150800C630008CDFF8301D4988884201D000F08BBE97
S3150800C640FFF723FE4FF6FF71884240F08486DFF835
S3150800C650B00BC07D062806D1FFF752FE4FF6FF71D4
S3150800C660884242D143E0DFF8980BC07D012840F0AC
S3150800C6707286DFF88C0B90F82200082840F06B864B
S3150800C6800020DFF87C1B81F82200DFF8740B808C11
S3150800C6904FF6F771884207DBDFF8640B808C0930A8
S3150800C6A0DFF85C1B888406E0DFF8540B808C0830C2
S3150800C6B0DFF84C1B8884DFF8480B408BDFF8401BFB
S3150800C6C0C883DFF83C0B808BDFF8341B0884DFF85F
S3150800C6D0940C0088DFF8281B4883DFF8880C40880C
S3150800C6E0DFF81C1B888300F032BE00F034BEDFF88A
S3150800C6F08C0C0500DFF8840CA8422BD3687E002832
S3150800C70026D0DFF8FC0A808CA988884220D1DFF879
S3150800C710F00A408CE98888421AD1DFF8E40A408B8F
S3150800C7202988884214D1DFF8D80A808B698888421C
S3150800C7300ED1DFF8A40905600020DFF8A4190870F7
S3150800C740DFF8BC0A90F82F00400700F145824CE25A
S3150800C7501E35CFE7DFF8A80A90F82F0010F03F0043
S3150800C760022829D1DFF8980A808CDFF8141C088083
S3150800C7700020DFF8101C0870DFF8080C0078002885
S3150800C7801AD1DFF8FC0B0088DFF8FC1BDFF8F42B66
S3150800C790127831F81210884206D1002005000020D0
S3150800C7A0DFF8E01B0870D6E0DFF8D80B0078401CED
S3150800C7B0DFF8D01B0870DFE7DFF8440A90F82F008F
S3150800C7C0400700F1C8851420DFF8341A81F82F00D5
S3150800C7D02820DFF8241A08805020DFF8241A81F868
S3150800C7E02E00DFF81C0A90F82900DFF8981B08705D
S3150800C7F0DFF80C0A90F82D00DFF8041A81F82900F2
S3150800C800DFF8800B0078DFF8F81981F82D00DFF8DB
S3150800C810F00990F82800DFF86C1B0870DFF8E009CB
S3150800C82090F82C00DFF8D81981F82800DFF8540BA7
S3150800C8300078DFF8CC1981F82C00DFF8C40990F8E5
S3150800C8402700DFF8401B0870DFF8B40990F82B00C2
S3150800C850DFF8AC1981F82700DFF8280B0078DFF835
S3150800C860A01981F82B00DFF8980990F82600DFF860
S3150800C870141B0870DFF8880990F82A00DFF8801979
S3150800C88081F82600DFF8FC0A0078DFF8741981F8C9
S3150800C8902A00DFF86C0990F82D00401CDFF86019B3
S3150800C8A081F82D00DFF8580990F82D00002826D1C8
S3150800C8B0DFF84C0990F82C00401CDFF8441981F881
S3150800C8C02C00DFF83C0990F82C00002817D1DFF877
S3150800C8D0300990F82B00401CDFF8241981F82B004A
S3150800C8E0DFF81C0990F82B00002808D1DFF810099A
S3150800C8F090F82A00401CDFF8081981F82A00DFF8AA
S3150800C9000009408CDFF8781A0880DFF8F408808C74
S3150800C910DFF8EC184884DFF8680A0088DFF8E018C2
S3150800C9208884DFF8DC08408BDFF8D418C883DFF882
S3150800C930D008808BDFF8C8180884DFF8280A008832
S3150800C940DFF8BC184883DFF81C0A4088DFF8B018FF
S3150800C950888300F0B9BCDFF82C0A007800283ED19D
S3150800C960DFF8180ADFF81C1A09781E225143084412
S3150800C970407E002809D1DFF8040ADFF8081A09788A
S3150800C9801E2251430844050029E0DFF8F009DFF8C4
S3150800C990F41909781E2251430844407E072816D107
S3150800C9A0002D0BD0A87EDFF8D419DFF8D829127825
S3150800C9B01E235A431144897E884208D2DFF8BC09EF
S3150800C9C0DFF8C01909781E22514308440500DFF82C
S3150800C9D0B4090078401CDFF8AC190870BBE7002DD5
S3150800C9E000F0B984DFF8F00605600320A876A87E73
S3150800C9F028760020A8750420E8750020E876DFF878
S3150800CA000008808CA880DFF8F807408CE880DFF8FB
S3150800CA10F007408B2880DFF8E807808B68800120C4
S3150800CA206876DFF8D00700782873DFF8C8074078FB
S3150800CA306873DFF8C0078078A873DFF8B807C0788E
S3150800CA40E87301202882DFF8B80790F82900E87211
S3150800CA50DFF8AC0790F82800A872DFF8A40790F86A
S3150800CA6027006872DFF8980790F8260028720120D8
S3150800CA70FFF793FCDFF8880790F82E0010F0F00017
S3150800CA8051287CDB0020DFF8FC180870DFF8F40872
S3150800CA900078DFF86C1791F82E10C9B20909C9B2E7
S3150800CAA0491FB0EB810F6ADADFF85407DFF8D418AC
S3150800CAB00978084490F83600DFF8D0180870DFF8CF
S3150800CAC0CC08007800285AD0DFF8C008007801287A
S3150800CAD007D1DFF8B0080078401CDFF8A8180870FE
S3150800CAE0D4E7DFF8A808007802282ED1DFF8100767
S3150800CAF0DFF890180978084490F83700042824D1FC
S3150800CB00DFF8FC06DFF87C180978084490F8380046
S3150800CB10DFF8EC16DFF86C281278114491F8391012
S3150800CB2051EA0020DFF858180880DFF85408008812
S3150800CB3040F20B61884202DB40F20A6002E0DFF84D
S3150800CB40400800886882A88219E0DFF8B406DFF892
S3150800CB5034180978084490F8370000280FD0DFF811
S3150800CB6024080078DFF89816DFF818281278114498
S3150800CB7091F837100818DFF80C18087086E71020A7
S3150800CB80DFF87C1681F82F00DFF8740690F82F007E
S3150800CB9050F00200DFF8681681F82F000220DFF84F
S3150800CBA0601681F836000420DFF8541681F837003D
S3150800CBB00620DFF84C1681F838000A20DFF8401600
S3150800CBC081F839002C20DFF8301608806020DFF85D
S3150800CBD0301681F82E002AE3002068762020DFF838
S3150800CBE00015087000F026FCB5E3DFF8140690F887
S3150800CBF02E00C0B200098000DFF888170870DFF839
S3150800CC00F8050088DFF87C170978401A1438DFF829
S3150800CC10E8150880687E10F00F00022807D1DFF8B3
S3150800CC20E00590F82F0010F03F00122828D0DFF812
S3150800CC30C8050088002806D1DFF8C40590F82F003B
S3150800CC40032108421CD0DFF8B80590F82600297A97
S3150800CC50884214D1DFF8A80590F82700697A884237
S3150800CC600DD1DFF89C0590F82800A97A884206D1EC
S3150800CC70DFF88C0590F82900E97A884200D0CBE2E3
S3150800CC80DFF87C0590F82F00C00665D5288A0028AD
S3150800CC9062D0298A15F10C00FFF778FADFF86005EB
S3150800CCA090F82A00DFF8E8160978884254D1DFF8A8
S3150800CCB0500590F82B00DFF8D816497888424BD1F2
S3150800CCC0DFF83C0590F82C00DFF8C416897888420E
S3150800CCD042D1DFF82C0590F82D00DFF8B416C97894
S3150800CCE0884239D1DFF8A80600782873DFF8A0064D
S3150800CCF040786873DFF898068078A873DFF890069E
S3150800CD00C078E873E87E00281ED195F9181095F9C1
S3150800CD101A20891A0800A97DC9B2B0EBD100A97DED
S3150800CD204118A97540B2002801D540B24042E97DB4
S3150800CD30C9B2B0EB9100E97D4118E975A97DC9B280
S3150800CD40EA7D12EBD10129760120DFF894130870E9
S3150800CD50287EA87600202882687E10F00F00C0B2D0
S3150800CD60012813D0C0F05782032800F0F48032D38C
S3150800CD70052800F02082C0F0ED81072800F04282E5
S3150800CD80C0F04182082800F0D98144E2DFF8500358
S3150800CD900078C0071ED5032068764020DFF84013C8
S3150800CDA0087000202882DFF85004008800280AD07E
S3150800CDB0CB48007850F00200C9490870DFF83804FB
S3150800CDC00088FFF7EAFA0020DFF83014088000F040
S3150800CDD031FB47E1BFE2C2480078C00740F1B180A5
S3150800CDE0DFF81C0490F82F0010F03F00122840F0DE
S3150800CDF0A880DFF80C0490F82E0010F0F0005128F7
S3150800CE007CDB0020DFF87C150870DFF878050078F1
S3150800CE10DFF8EC1391F82E10C9B20909C9B2491FF7
S3150800CE20B0EB810F6ADADFF8D803DFF8581509780E
S3150800CE30084490F83600DFF854150870DFF84C05FA
S3150800CE40007800285AD0DFF844050078012807D171
S3150800CE50DFF830050078401CDFF828150870D4E79D
S3150800CE60DFF82805007802282ED1DFF89403DFF8CA
S3150800CE7014150978084490F83700042824D1DFF8F7
S3150800CE808003DFF800150978084490F83800DFF8C1
S3150800CE907013DFF8F0241278114491F8391051EA2A
S3150800CEA00020DFF8DC140880DFF8D404008840F29C
S3150800CEB00B61884202DB40F20A6002E0DFF8C00438
S3150800CEC000886882A88219E0DFF83403DFF8B41412
S3150800CED00978084490F8370000280FD0DFF8A40432
S3150800CEE00078DFF81C13DFF89C241278114491F8B7
S3150800CEF037100818DFF88C14087086E70320687660
S3150800CF00BF4890F826002872BD4890F82700687236
S3150800CF10BB4890F82800A872B94890F82900E8722A
S3150800CF200120FFF73AFA42206D490870002028824E
S3150800CF300020B14908800020B049088000F07AFA3C
S3150800CF4090E020206649087000F074FA00206249D3
S3150800CF500968487630E4AA4890F82F00C00729D512
S3150800CF60687EC00626D4288A002840F0F481A248A4
S3150800CF700088401C80B2FFF710FA5948007850F034
S3150800CF801000574908709C480088002805D0544866
S3150800CF90007850F002005249087000F04BFA012060
S3150800CFA02882082068760020E8761120944981F8BE
S3150800CFB02F0035E1924890F82F00800619D54F4882
S3150800CFC000688F4991F834108D4A92F8352052EA54
S3150800CFD0012108444949086087480088884991F82A
S3150800CFE03410874A92F8352052EA0121401A8249BC
S3150800CFF008808148008800280CD0687EC00609D4BD
S3150800D0003748007850F00200354908707A48008899
S3150800D010FFF7C3F97A4890F830000002784991F88A
S3150800D02031104018DFF858130880A88ADFF8501323
S3150800D0300988884204D3DFF848030088002803D10A
S3150800D040A88ADFF83C130880DFF834030088688272
S3150800D05023480078032108426FD0002067490880DA
S3150800D06000F0E8F91E480078800609D500206349D3
S3150800D0700880002068761420614981F82F00CFE0E7
S3150800D08017480078C0060DD500205C4908800120A5
S3150800D0902882042068760020E8761120584981F80D
S3150800D0A02F00BDE05548008800281ED00C4800789F
S3150800D0B0C00701D500202882288A002812D1688A4C
S3150800D0C04E490988884202D2688A4C4908804B48EA
S3150800D0D00088288209E000BFC01C00204E080020F6
S3150800D0E0DF1C0020288A454908800020E876044885
S3150800D0F0006802490860414804E000BFB81C0020E7
S3150800D100BC1C0020008800280BD0288A002808D0DC
S3150800D110288A2830384908801820394981F82F008C
S3150800D12081E09C480078800707D528203249088086
S3150800D1301020334981F82F0075E00CE195480078F6
S3150800D140C00706D50020687610209249087000F0BE
S3150800D15071F960E028480088002803D0264800882E
S3150800D160FFF71BF9264890F82F00C00715D5894800
S3150800D1700078C00706D5072068760020A876002024
S3150800D180288201E0062068760120FFF706F91020BC
S3150800D1908049087000F04EF93EE07E480078C007E6
S3150800D1A004D50520687600202882D4E01248008835
S3150800D1B0002831D1CFE010480088002803D00E4857
S3150800D1C00088FFF7EAF80E4890F82F00C0070CD53C
S3150800D1D0072068760020A8760120FFF7DEF81020E1
S3150800D1E06C49087000F026F916E003480088002804
S3150800D1F012D1B0E0C41C0020D01C0020D21C002094
S3150800D2001808002008E063480078C00703D50720FF
S3150800D21068760020A8769EE010205F4981F82F00E6
S3150800D22028205E49088050205B4981F82E00287A1C
S3150800D230594981F82A00687A574981F82B00A87A53
S3150800D240554981F82C00E87A534981F82D00287B46
S3150800D250514981F82600687B4F4981F82700A87B49
S3150800D2604D4981F82800E87B4B4981F829000620BA
S3150800D2704949C875A88848494884E8884649888439
S3150800D2803848008844494883364840884249888354
S3150800D29028884149C88368883F490884687EC0064B
S3150800D2A00AD500203C4981F831003B4890F8310006
S3150800D2B0394981F8300007E00620374981F83000FF
S3150800D2C00A20354981F831004020334988753348AA
S3150800D2D0008880B2000A30490874304800882E4910
S3150800D2E0487400202C4981F835002B4890F8350001
S3150800D2F0294981F83400002027494886FFF700F8B5
S3150800D300C043254948864520234988730020224979
S3150800D310C8730020204948751F48407D1E49087576
S3150800D3201F480088401C1E4908801D48008880B296
S3150800D330000A194988741A4800881749C8740020D1
S3150800D34015490883FEF7A1FFC04313490883002047
S3150800D3501049087005E000201049088000200D4992
S3150800D360087031BDAC1C0020FCF30008010089B22E
S3150800D370090A51EA002080B270470000801B00208D
S3150800D380DA1C0020E01C0020D41C0020E11C002030
S3150800D390C81C0020DF1C002018080020D01C002014
S3150800D3A0D61C002080B500F0DDF800F0EFFA10F585
S3150800D3B0FA706149086000F0E9FA00F51C5010306F
S3150800D3C05E490860FEF7A1FF4FF6A960ADF80000B8
S3150800D3D043F61370ADF80200BDF8000058490880FE
S3150800D3E0BDF80200564948804FF6FF70ADF80000B8
S3150800D3F00020ADF80200BDF8000052490880BDF8CB
S3150800D4000200504948804FF6A960ADF8000040F286
S3150800D4101310ADF80200BDF800004B490880BDF8AE
S3150800D4200200494948804EF60300FEF79BFF00F0CC
S3150800D43077F901BD10B54548007840060FD4434832
S3150800D440007880070BD5424800680400241D207820
S3150800D450FF2804D16078002801D100F0C8FA10BD71
S3150800D46038B500F08AF90500002D2DD03948058019
S3150800D4704FF40060FFF77AFF3749898980B2814205
S3150800D4800ED10120FEF7BCFF3248008800281BD0C9
S3150800D49000F0BDFD00F090F900202E49088013E049
S3150800D4A040F60600FFF762FF2B49898980B2814260
S3150800D4B00AD100F032FD27480088002804D000F081
S3150800D4C07BF900202349088000F060FA1A490968A8
S3150800D4D0884220D31848006810F5FA701649086083
S3150800D4E000200400002C16D11C481E2101FB04F163
S3150800D4F008441B4908600220FEF782FF1548008889
S3150800D500002806D000F083FD00F056F900201149E6
S3150800D5100880641CE6E700F039FA08490968884279
S3150800D52008D30648006800F51C5010300349086007
S3150800D53000F00AFC31BD0000A01C0020A41C00203D
S3150800D540AC1C0020B41C0020B01C0020DF1C0020EE
S3150800D550B81C0020D01C002018080020801B0020C2
S3150800D560C01C002010B5B2B001215FF0F05000F0E9
S3150800D570C9FE0121472000F0C5FE01214FF4804075
S3150800D58000F0DEFE012000F01DFF8E200090002036
S3150800D5908DF8060002208DF8040000208DF807009B
S3150800D5A002208DF805006946CA4800F011FF0B22D3
S3150800D5B00121C84800F065FF0B220221C54800F08A
S3150800D5C060FF0B220321C34800F05BFF0B220721F3
S3150800D5D0C04800F056FF4FF40060009000208DF818
S3150800D5E0060002208DF8040000208DF807000220AE
S3150800D5F08DF805006946B84800F0EAFE0B220B21B3
S3150800D600B54800F03EFF3220009000208DF8060055
S3150800D61002208DF8040000208DF8070002208DF8FE
S3150800D62005006946AD4800F0D3FE0B220121AB4840
S3150800D63000F027FF0B220421A84800F022FF0B2246
S3150800D6400521A64800F01DFF4FF4C04000900020B9
S3150800D6508DF8060002208DF8040000208DF80700DA
S3150800D66002208DF8050069469B4800F0B1FE0B22A2
S3150800D6700D21994800F005FF0B220E21964800F06F
S3150800D68000FF00F02BFF01F0B7F901F0BEF9012801
S3150800D690FBD003A801F092F80020039000200A901E
S3150800D6A04FF400700D9000200E905FF0004011902E
S3150800D6B02020149000201690002017900020189023
S3150800D6C04FF400600B904FF480400890002004004F
S3150800D6D0202C18D20221200080B201F0F4F8ADF80F
S3150800D6E00A000321200080B201F0EDF8ADF8080029
S3150800D6F002987B49884203D002987A49884200D129
S3150800D70001E0641CE4E7210089B203A800F0F2FEF8
S3150800D71000F0CAF800F09EF801F0C5F832B010BD66
S3150800D72082B008208DF8000000208DF8010027201F
S3150800D7308DF8020069208DF803005B208DF804003F
S3150800D74045208DF805009DF80000674908709DF88A
S3150800D7500100654948709DF80200634988709DF884
S3150800D76003006149C8709DF804005F4908719DF877
S3150800D77005005D49487102B0704770B55B4800689E
S3150800D780C00F002816D159480068C0F30D400400A0
S3150800D790574D584E22002900300001F095F953489C
S3150800D7A0006850F00040514908600120524908605D
S3150800D7B0200000E0002070BD70B550480068C00F1A
S3150800D7C00028FAD14E4804884A4D4E4E22002900B8
S3150800D7D0300001F079F94B484849886000204749EC
S3150800D7E008604648006850F4801044490860434879
S3150800D7F0006850F00050414908604048006850F001
S3150800D80080503E4908603D48006830F000603B495A
S3150800D81008603A48006830F080603849086000209F
S3150800D82036494860364800883449496860F30B0130
S3150800D830324841603148406830F480502F4948608A
S3150800D8402E48006850F000402C49086001202E49F7
S3150800D850086070BD2648254988600020234908606D
S3150800D86022482249C8600020204948601F4840686D
S3150800D87030F400401D4948601C48406850F4804018
S3150800D8801A4948604FF4C8601849496860F30C01A2
S3150800D890164841601548006850F000401349086072
S3150800D8A012481A4908607047164814498860134890
S3150800D8B01249C8601148006850F480100F49086082
S3150800D8C000200E49086000200C4948600B481049A2
S3150800D8D00860704700000240001802400008024035
S3150800D8E019162200F1C00700901C0020001C002019
S3150800D8F05C0E00201808002008900240801C0020BA
S3150800D900D01C00209C140020049002400C90024079
S3150800D9101090024010B440B2002808D50A01204BE6
S3150800D92040B210F00F04234403F8042C03E00A0164
S3150800D9301C4B40B21A5410BC704710B50400B4F121
S3150800D940807F01D3012010E024F07F40401E164955
S3150800D95008600F215FF0FF30FFF7DCFF0020134956
S3150800D9600860072012490860002010BD80B51148DC
S3150800D97000684FF47A71B0FBF1F0FFF7DEFF002084
S3150800D98000F001F801BD0C49086070470A480068B4
S3150800D990704709480068401C07490860704700003E
S3150800D9A018ED00E000E400E014E000E018E000E014
S3150800D9B010E000E010000020A81C0020BFF34F8FE5
S3150800D9C0D648006810F4E060D5490843D349086092
S3150800D9D0BFF34F8FFEE780B500F00DF800F0F5F8BD
S3150800D9E001BD80B500F052F800F06FF901BD80B5B1
S3150800D9F0FFF7E4FF01BD00B587B00121202000F044
S3150800DA009FFC0121042000F07DFC08220621C54860
S3150800DA1000F037FD08220721C24800F032FD002039
S3150800DA208DF8060001208DF8070002208DF8040005
S3150800DA304020009002208DF805006946B94800F09C
S3150800DA40C7FC02208DF80400802000906946B5487E
S3150800DA5000F0BEFC4FF4614002900020ADF80C00C7
S3150800DA600020ADF80E000020ADF810000020ADF83B
S3150800DA7014000C20ADF8120002A9AB4801F060F8BA
S3150800DA800121A94801F0DAF807B000BD80B5A7481A
S3150800DA900078002813D1A64800F03EF801283AD1AC
S3150800DAA0A3480078002836D0FFF770FFA149086020
S3150800DAB001209E49087000209F4908702BE09C4869
S3150800DAC09D4909780844401C00F026F8012818D119
S3150800DAD099480078401C98490870974800789449F6
S3150800DAE00978884217D100209049087090484078F4
S3150800DAF0FF2810D18E48807800280CD1FFF777FFD1
S3150800DB0009E0FFF743FF8B4909686431814202D275
S3150800DB1000208649087001BD10B5040020218248FE
S3150800DB2001F09EF8012805D17F4801F095F820708C
S3150800DB30012000E0002010BDF0B40400002005001C
S3150800DB40EDB2122D3ED24AF21040A4B27B4EEDB28F
S3150800DB5016F81560794FEDB207EB45077F78BE19C1
S3150800DB60761C06FB04F690FBF6F706FB1700002862
S3150800DB7026D14AF21040A4B2704EEDB216F81560DE
S3150800DB806E4FEDB207EB45077F78BE19761C06FB8C
S3150800DB9004F690FBF6F008800888002810D008885C
S3150800DBA0B0F5806F0CDC6548EDB210F81500107002
S3150800DBB06248EDB200EB450040781870012002E09B
S3150800DBC06D1CBDE70020F0BC704700B58BB0012185
S3150800DBD0022000F097FB09220521594800F051FC64
S3150800DBE009220621564800F04CFC602004900220C9
S3150800DBF08DF8140002208DF8150000208DF8160007
S3150800DC0001208DF8170004A94D4800F0E1FB012119
S3150800DC105FF0C06000F085FB4A4801F031F801A8C2
S3150800DC2001F05FF96B460DF101020DF102014FF4A7
S3150800DC30FA70FFF781FF00208DF80A0000208DF8A2
S3150800DC400B0000208DF80C0000208DF80D00002038
S3150800DC508DF80E0000208DF80F0000208DF80600C4
S3150800DC6000208DF807009DF80100401E8DF8080079
S3150800DC709DF80000401E8DF80900BDF80200ADF8B9
S3150800DC80040001A92F4801F017F80E208DF822008C
S3150800DC9000208DF8230001208DF824000020ADF81F
S3150800DCA018000020ADF81A000020ADF81C0000206E
S3150800DCB0ADF81E000020ADF8200001208DF82500E3
S3150800DCC006A801F085F80BB000BD10B586B0002493
S3150800DCD000211C4801F090F900281CD06A46002152
S3150800DCE0184801F015F99DF80800002806D1009893
S3150800DCF040F26761884201D101200400E4B2012C98
S3150800DD0009D19DF80B00FF2805D19DF80C000028C5
S3150800DD1001D1FFF76CFE06B010BD00000CED00E067
S3150800DD200400FA050008024000140140DD1C00202A
S3150800DD303C1B0020981C0020DC1C002030F3000847
S3150800DD40000402400068004070B5DFF870040078EF
S3150800DD50401CDFF8681408700020DFF858140870B3
S3150800DD60DFF850040078082823DADFF84C04DFF8D7
S3150800DD70441409780C225143084404002088618819
S3150800DD80084300280DD0DFF834040078A17A401A39
S3150800DD90782806DB0425002632002900200001F039
S3150800DDA04FF9DFF810040078401CDFF808140870F3
S3150800DDB0D6E770BD2DE9F84304000D000020DFF812
S3150800DDC0F4130870DFF8EC03007808282BDADFF87C
S3150800DDD0E803DFF8E01309780C22514308440600EB
S3150800DDE03088002817D07088002814D020883188F9
S3150800DDF0884210D16088718888420CD1062716F1AE
S3150800DE0004083A002900404600F05EFEDFF8AC033D
S3150800DE100078B0727FE0DFF89C030078401CDFF8DA
S3150800DE2094130870CEE70020DFF888130870DFF82F
S3150800DE3084030078082816DADFF87C03DFF8741301
S3150800DE4009780C225143084406003088002802D17C
S3150800DE507088002807D0DFF85C030078401CDFF8DC
S3150800DE6054130870E3E7DFF84C030078082840D11C
S3150800DE700020DFF84C1308700020DFF848130870FC
S3150800DE800020DFF830130870DFF828030078082828
S3150800DE9024DADFF82403DFF81C1309780C2251432F
S3150800DEA008440600DFF818030078DFF8101309782D
S3150800DEB0B27A891A88420BDADFF800030078B17A59
S3150800DEC0401ADFF8FC120870BA480078BD49087095
S3150800DED0B8480078401CB7490870D5E7B9480078B3
S3150800DEE0B4490870B448B34909780C225143084428
S3150800DEF0060004273A002100300000F0E5FD5FF037
S3150800DF00060816F1040942462900484600F0DCFDD9
S3150800DF10AA480078B072BDE8F1832DE9F84FAA48FF
S3150800DF2000882A2803D20020A74908806DE000202F
S3150800DF30A5490880A548808AB0F5807F03D0B0F54A
S3150800DF40007F52D061E0A148C08CA1490988884267
S3150800DF504AD19E48008D9E494988884244D19D49A8
S3150800DF609D48FFF727FF4FF40070984988820620DE
S3150800DF700090984C994D009A2100280000F0A4FDC5
S3150800DF800625974E934F2A003100380000F09CFD75
S3150800DF900627DFF84C82DFF84C923A00414648469D
S3150800DFA000F092FD5FF00609DFF830A2DFF81CB238
S3150800DFB04A465146584600F087FD8448808B834977
S3150800DFC0C8848248C08B81490885814800887F4972
S3150800DFD088837F4840887D49C8834FF4C1607B4960
S3150800DFE088812A20784908800FE07848C08C7849CB
S3150800DFF00988884209D17548008D7549498888423B
S3150800E00003D174497448FFF7D5FEBDE8F18F2DE9B1
S3150800E010F04F83B06D48C08B7349098888420ED18A
S3150800E0206A48008C70494988884208D106246F4D91
S3150800E030664E22002900300000F046FDA7E063483E
S3150800E040C08B6B490988084061490988684A128863
S3150800E050114088420BD15D48008C654949880840C3
S3150800E0605B494988624A52881140884208D061480B
S3150800E0700088614908805F4840885F49488007E012
S3150800E0805248C08B5C4908805048008C5A494880E1
S3150800E09000204849087047480078082818DA464892
S3150800E0A0444909780C225143084400905248008894
S3150800E0B000990988884205D14F48408800994988BF
S3150800E0C0884205D03B480078401C3A490870E2E788
S3150800E0D038480078082851D106200190FF243B4D86
S3150800E0E022000199280000F0ABFF062500263B4FC9
S3150800E0F032002900380000F0A3FF0627DFF8E08089
S3150800E100DFF8E0903A004146484600F0DDFC5FF053
S3150800E1100609DFF8CCA0DFF8BCB04A465146584697
S3150800E12000F0D2FC344800882849C8843248408820
S3150800E1302649088526480088244988832448408833
S3150800E1402249C8834FF48070204988824FF4807032
S3150800E1501E49C88108201D49088206201B49887463
S3150800E16004201A49C8744FF4C160184988812348A5
S3150800E170234908602A201449088018E006240098D4
S3150800E180051D124E22002900300000F09DFC0624D1
S3150800E190134D144E22002900300000F095FC08208B
S3150800E1A00A498881084800880E3007490880BDE872
S3150800E1B0F78F0000E21C0020DC1A0020E41C002077
S3150800E1C0E51C0020E31C0020D01C002018080020B5
S3150800E1D0AC1C00202E080020340800203808002037
S3150800E1E0901C00201E08002000F40008F4F3000824
S3150800E1F0B41C0020B01C0020CC1C00204E080020B7
S3150800E200B81C0020F0B400210022002302240025B7
S3150800E2100226DFF888713F6817F00C0739000F00EF
S3150800E220002F04D0042F06D0082F08D03CE0DFF8D2
S3150800E230747107603BE0DFF87071076037E0DFF85C
S3150800E24060713F68C7F380573D00DFF854713F6837
S3150800E25017F03F073E00002D0DD0DFF84C71B7FBD5
S3150800E260F6F7DFF83CC1DCF800C0CCF3881C0CFBE1
S3150800E27007F73B000CE0DFF82C71B7FBF6F7DFF881
S3150800E28020C1DCF800C0CCF3881C0CFB07F73B0068
S3150800E290DFF80C713F68C7F301477F1C7F003C001D
S3150800E2A0B3FBF4F7076002E0DFF8F8700760DFF801
S3150800E2B0EC703F6817F0F00739000909DFF8EC70D1
S3150800E2C07F5C3A000768D7404760DFF8D0703F6840
S3150800E2D017F4E0573900890ADFF8D0707F5C3A00F6
S3150800E2E04768D74087602D4F3F6817F46047390065
S3150800E2F0490BDFF8B8707F5C3A004768D740C760BB
S3150800E300F0BC7047C9B2002905D0294A12680243F1
S3150800E310274B1A6004E0264A12688243244B1A6087
S3150800E3207047C9B2002905D0224A12680243214B18
S3150800E3301A6004E01F4A126882431E4B1A6070472F
S3150800E340C9B2002905D01C4A126802431A4B1A6042
S3150800E35004E0194A12688243174B1A607047C9B21B
S3150800E360002905D0154A12680243144B1A6004E0C6
S3150800E370124A12688243114B1A607047C9B20029C3
S3150800E38005D00F4A126802430D4B1A6004E00C4A86
S3150800E390126882430A4B1A60704700000838024028
S3150800E3A0043802400024F400001BB70000000020D7
S3150800E3B030380240403802404438024010380240A3
S3150800E3C0203802400149086070470000DC002742F7
S3150800E3D0F0B400220023002400252A00102A4AD27D
S3150800E3E0012595402B000D681D402C009C4240D10C
S3150800E3F0056803261700FFB27F00BE40B5430560D7
S3150800E40005680E791700FFB27F00BE4035430560E8
S3150800E4100D79012D02D00D79022D1AD185680326B2
S3150800E4201700FFB27F00BE40B543856085684E7908
S3150800E4301700FFB27F00BE40354385604568012658
S3150800E4409640B543456045688E799640B6B23543E1
S3150800E4504560C56803261700FFB27F00BE40B54376
S3150800E460C560C568CE791700FFB27F00BE40354348
S3150800E470C560521CB2E7F0BC704701837047418300
S3150800E4807047F0B400230024D2B211F00705EDB2AC
S3150800E490AD0012FA05F52B0089B2CD1000EB850503
S3150800E4A089B2CE1000EB8606366A0F2711F0070CE4
S3150800E4B05FFA8CFC5FEA8C0C17FA0CF7BE432E62E7
S3150800E4C089B2CD1000EB85052D6A1D432C0089B253
S3150800E4D0CD1000EB85052C62F0BC704780B5012194
S3150800E4E05FF00070FFF73BFF00215FF00070FFF759
S3150800E4F036FF01BD2DE9F04186B004000D00002667
S3150800E5005FF0000800200190DFF8187500200090E1
S3150800E510DFF824050068804638F01C0802A8FFF7D3
S3150800E52071FE03980700DFF81405874206D3DFF863
S3150800E5301005874202D258F0080814E0DFF80005F3
S3150800E540874206D3DFF8FC04874202D258F00C084B
S3150800E55009E0DFF8F004874203D3DFF810058742A5
S3150800E56001D358F00408DFF8D004C0F800804FF44F
S3150800E57000420021280080B200F0DCF9002801D111
S3150800E580002018E15FF0806001900198002803D010
S3150800E5900198401E0190F8E72068002851D000989D
S3150800E5A0401C00900121280080B200F08CF9400739
S3150800E5B004D40098DFF8E4148842F0D30098DFF812
S3150800E5C0DC14884201D10020F5E0002000904FF4C9
S3150800E5D080520021280080B200F0ACF9002801D151
S3150800E5E00020E8E00098401C00900121280080B235
S3150800E5F000F069F9800604D40098DFF8A014884270
S3150800E600F0D30098DFF89414884201D10020D2E0B4
S3150800E610002000901021280080B200F054F906006E
S3150800E620700703D54FF40060206201E000202062E5
S3150800E630B00702D5002060611CE04FF4804060619D
S3150800E64018E0206A6169490851EAD00292B20021AD
S3150800E650280080B200F06EF9002801D10020AAE057
S3150800E6607FF07F4001900198002803D00198401E52
S3150800E6700190F8E7DFF81C0400688046DFF8180404
S3150800E68010EA08086068A1680843E1680843216938
S3150800E690084361690843A1690843E1690843216A97
S3150800E6A00843616A0843A16A0843E16A0843216B83
S3150800E6B00843616B084350EA0808DFF8D803C0F836
S3150800E6C00080A06BE16B0843216C0843616C08432A
S3150800E6D0A16C0843E16C0843216D0843616D08434A
S3150800E6E0DFF8BC130860A06DDFF8B8130860E06DAA
S3150800E6F0DFF8B4130860DFF8B403006880464FF605
S3150800E700417010EA0808206E616E51EA0040A16E59
S3150800E7100843E16E0843216F0843616F084350EAD6
S3150800E7200808DFF88803C0F80080A06FE16F084387
S3150800E730DFF87C130860DFF87C0300688046DFF8A2
S3150800E740780310EA0808D4F88000D4F8841008433F
S3150800E750D4F888100843D4F88C100843D4F89010DD
S3150800E7600843D4F894100843D4F898100843D4F80A
S3150800E7709C100843D4F8A010084350EA0808DFF8AC
S3150800E7803403C0F80080D4F8A400D4F8A8100843CD
S3150800E790D4F8AC100843D4F8B0100843D4F8B41031
S3150800E7A050EA8100D4F8B810084350F40000DFF8A6
S3150800E7B00C130860012006B0BDE8F0810021016055
S3150800E7C000214160002181600021C16000210161B2
S3150800E7D000214161002181610021C161002101629E
S3150800E7E000214162002181620021C162002101638A
S3150800E7F000214163002181630021C1634021016436
S3150800E80020214164002181640021C1640021016541
S3150800E81000214165002181650021C165002101664D
S3150800E82080214166002181660021C16600210167B9
S3150800E83000214167002181670021C1675FF080617F
S3150800E840C0F880105FF00071C0F884105FF0807126
S3150800E850C0F888105FF40011C0F88C100021C0F8C9
S3150800E86090100021C0F894100021C0F898100021DB
S3150800E870C0F89C100021C0F8A0105FF00071C0F825
S3150800E880A4100021C0F8A8105FF40031C0F8AC103D
S3150800E8904FF48071C0F8B0100021C0F8B410002100
S3150800E8A0C0F8B810704780B5012000F07BF800F07A
S3150800E8B0BBF8012000F08BF8012000F0C5F8012014
S3150800E8C000F0D6F801BD18B402000023002000901D
S3150800E8D0DFF864010068030013F01C0392B2D0024B
S3150800E8E010F47840034389B2880110F4F8600343B2
S3150800E8F033F0020353F00103DFF83C01036000988C
S3150800E900401C0090DFF8300100680300D80704D5E2
S3150800E9100098DFF88841A042F1D30098DFF87C41DF
S3150800E920A04201D1002003E0DFF89401006880B21C
S3150800E93012BC704738B40300002400200090DFF8AA
S3150800E940F8000068040014F01C049BB2D80210F406
S3150800E9507840044389B2880110F4F860044354F0FF
S3150800E960020454F0010492B2DFF854010260DFF8A1
S3150800E970C80004600098401C0090DFF8BC000068DE
S3150800E9800400E00704D50098DFF81051A842F1D337
S3150800E9900098DFF80851A84201D1002000E00120C4
S3150800E9A032BC7047C0B2002808D0DFF8E810096802
S3150800E9B051F00801DFF8DC20116007E0DFF8D41019
S3150800E9C0096831F00801DFF8CC2011607047C0B241
S3150800E9D0002808D0DFF8BC10096851F00401DFF8F8
S3150800E9E0B420116007E0DFF8AC10096831F00401C3
S3150800E9F0DFF8A02011607047DFF8C800006850F003
S3150800EA000100DFF8C010086070470020DFF8B41076
S3150800EA100968C90702D50121080001E0002108009C
S3150800EA20C0B27047000E27072248006850F48010CD
S3150800EA30204908607047000010800240002D31010F
S3150800EA40C00E160200879303C0B2002806D01949E3
S3150800EA50096851F40051174A116005E0154909681B
S3150800EA6031F40051134A11607047000001E1F505C1
S3150800EA70C0B2002806D00F49096851F002010D4AB4
S3150800EA80116005E00B49096831F00201094A116075
S3150800EA9070470000008002400F8120FFFFFF04003E
S3150800EAA004800240088002400C8002401880024020
S3150800EAB01C80024018900240233FDEF80090024076
S3150800EAC0148002400090024062B38B0708D0521EA1
S3150800EAD011F8013B00F8013B00F024808B07F6D1C2
S3150800EAE0830740F0208000BF103A07D330B4B1E85E
S3150800EAF03810103AA0E83810F9D230BC530724BFB2
S3150800EB00B1E80810A0E8081044BF51F8043B40F8E3
S3150800EB10043BD20724BF31F8022B20F8022B44BF4E
S3150800EB200B7803707047083A07D3B1E80810083A1B
S3150800EB3040F8043B40F804CBF7D25307E4E700005B
S3150800EB402DE9F04385B004000D005FF000090026AA
S3150800EB5000275FF00008A8890028208A814639F432
S3150800EB604059E88850EA0909A4F81090A089814616
S3150800EB70314810EA0909A888298908436989084398
S3150800EB8050EA0909A4F80C90A08A814639F440791C
S3150800EB90A88950EA0909A4F814906846FFF732FBD9
S3150800EBA02348844202D02348844202D103980600AF
S3150800EBB001E002980600A089000408D5192000FB88
S3150800EBC006F029684900B0FBF1F0070007E01920B4
S3150800EBD000FB06F029688900B0FBF1F00700642005
S3150800EBE0B7FBF0F0000181465FEA1910642101FBCA
S3150800EBF010708046A08900040AD55FEAC800323042
S3150800EC006421B0FBF1F010F0070050EA090909E0A9
S3150800EC105FEA081032306421B0FBF1F010F00F0003
S3150800EC2050EA0909A4F8089005B0BDE8F083000089
S3150800EC300010014000140140F3E9FFFFC9B20029A2
S3150800EC4004D0828952F40052828104E082894DF60A
S3150800EC50FF731A40828170478088C005C00D7047CF
S3150800EC600200002089B2B1F5007F13880B4202D05A
S3150800EC700123180001E000231800C0B27047000005
S3150800EC8010B50400DFF89C0384420AD101215FF025
S3150800EC900070FFF773FB00215FF00070FFF76EFB53
S3150800ECA009E001215FF08060FFF768FB00215FF053
S3150800ECB08060FFF763FB10BD30B40200002000231C
S3150800ECC0146834F002041460146854F001041460E3
S3150800ECD05468E40705D44FF6FF74A34201D05B1CC1
S3150800ECE0F6E75468E40702D4002420006DE08C7926
S3150800ECF0012C04D1146854F08004146003E01468ED
S3150800ED0034F080041460CC79012C04D1146854F0D2
S3150800ED104004146003E0146834F0400414600C7A6C
S3150800ED20012C04D1146854F02004146003E014681C
S3150800ED3034F0200414604C7A012C04D1146854F081
S3150800ED401004146003E0146834F0100414608C7A1C
S3150800ED50012C04D1146854F00804146003E0146804
S3150800ED6034F008041460CC7A012C04D1146854F0E9
S3150800ED700404146003E0146834F0040414608C7806
S3150800ED80CD782D0655EA84740D7954EA05444D79F3
S3150800ED9054EA05540D886D1E2C43D4611468640822
S3150800EDA064001460002423005468E40705D54FF670
S3150800EDB0FF74A34201D05B1CF6E75468E40702D54A
S3150800EDC00024200001E001242000C0B230BC7047B6
S3150800EDD010B400210122837A9A401100DFF84822F4
S3150800EDE0126852F00102DFF840321A60DFF83C225E
S3150800EDF012688A43DFF834321A60027B002A19D176
S3150800EE00DFF82C2212688A43DFF824321A60C28897
S3150800EE10438853EA0242DFF81C32847A43F83420E6
S3150800EE20DFF81022837A02EBC3028388048854EA47
S3150800EE3003435360027B012A19D1DFF8F4211268D3
S3150800EE400A43DFF8EC311A600288438853EA024223
S3150800EE50DFF8E031847A43F83420DFF8D821837A62
S3150800EE6002EBC3028388C48854EA03435360C27A18
S3150800EE70002A07D1DFF8C02112688A43DFF8B831C3
S3150800EE801A6006E0DFF8B02112680A43DFF8A831F5
S3150800EE901A600289002A06D1DFF8A02112688A437F
S3150800EEA0DFF898311A600289012A06D1DFF88C2129
S3150800EEB012680A43DFF884311A60427B012A06D1B8
S3150800EEC0DFF8682112680A43DFF860311A60DFF854
S3150800EED05821126852085200DFF84C311A6010BCEB
S3150800EEE07047002181710021C17100210172002142
S3150800EEF04172002181720021C172002181700021B6
S3150800EF00C1700321017102214171012101807047FD
S3150800EF10C9B20B010344D3F8B03113F004031372DA
S3150800EF20137A002B07D1C9B20B010344D3F8B031C9
S3150800EF305B0D136006E0C9B20B010344D3F8B03188
S3150800EF40DB085360C9B20B010344D3F8B03113F0A0
S3150800EF5002035372C9B20B010344D3F8B43113F058
S3150800EF600F039372C9B20B010344D3F8B4311B0AD9
S3150800EF70D374C9B20B010344D3F8B831D372C9B2FA
S3150800EF800B010344D3F8B8311B0A1373C9B20B013A
S3150800EF900344D3F8B8311B0C5373C9B20B010344AD
S3150800EFA0D3F8B8311B0E9373C9B20B010344D3F8D7
S3150800EFB0BC31D373C9B20B010344D3F8BC311B0A65
S3150800EFC01374C9B20B010344D3F8BC311B0C537438
S3150800EFD0C9B20B010344D3F8BC311B0E9374C9B2F2
S3150800EFE0002904D1C36853F02003C36003E0036912
S3150800EFF053F020030361704702000020C9B20029BC
S3150800F00004D1D36813F00303180009E0C9B2012933
S3150800F01004D1136913F00303180001E00023180054
S3150800F020C0B2704700640040006600401C6600409D
S3150800F0300C660040406600400466004014660040C6
S3150800F04062F30F2262F31F42401810F0030308D040
S3150800F050C91A1FD3DB0748BF00F8012D28BF20F8BF
S3150800F060022D130030B414461546103928BF20E97E
S3150800F0703C00FAD8490728BF20E90C0048BF40F8E9
S3150800F080042D890028BF20F8022D48BF00F8012D5D
S3150800F09030BC7047C91818BF00F8012DCB0728BF28
S3150800F0A000F8012D7047000080B54348006850F00D
S3150800F0B00100414908600020404908603E48006850
S3150800F0C03F4908403C4908603E483F4908603A487D
S3150800F0D0006830F480203849086000203B49086001
S3150800F0E000F001F801BD82B00020019000200090D8
S3150800F0F03148006850F480302F4908602E4800686F
S3150800F10010F4003000900198401C019000980028E7
S3150800F11003D10198B0F5A06FF0D1274800688003A5
S3150800F12002D50120009001E00020009000980128F7
S3150800F1303ED12748006850F0805025490860254888
S3150800F140006850F44040234908601C4800681B4981
S3150800F15008601A48006850F40040184908601748C3
S3150800F160006850F4A050154908601B481649086005
S3150800F1701148006850F080700F4908600E48006812
S3150800F1808001FBD540F20560144908600B48006809
S3150800F19080088000094908600848006850F00200A5
S3150800F1A0064908600548006810F00C000828F9D1DF
S3150800F1B002B07047000000000038024008380240DC
S3150800F1C0FFFFF6FE10300024043802400C380240D7
S3150800F1D040380240007000400C544007003C024092
S3150800F1E000B583B001210420FFF78CF84FF40050D6
S3150800F1F0009001208DF8040000208DF806000120FB
S3150800F2008DF8070002208DF8050069461548FFF7B6
S3150800F210DFF84FF400511348FFF72FF907BD10B573
S3150800F220FEF7B4FB040010480068201AB0F5FA7F10
S3150800F23016D30E480078002808D101200B4908701B
S3150800F2404FF400510748FFF71AF907E0002007496D
S3150800F25008704FF400510348FFF70FF9024804609D
S3150800F26010BD0000000802409C1C0020DE1C002087
S3150800F27019E050F8041BCB0744BFA9F1010359183C
S3150800F280121F0023042A41F8043BF9D25FEA827C64
S3150800F2900B4604D54FF0000CA1F800C09B1CD10703
S3150800F2A044BF0021197050F8042B002AE1D1704799
S3150800F2B080B500F00BF8FEF775F8FEF78CFBFFF744
S3150800F2C0AEFFFEF7CDF8FEF78CFBF8E780B5FFF743
S3150800F2D0EBFEFFF785FFFEF749FB01BD10B450F8BA
S3150800F2E0041B79B10268436802440830DC0744BF4E
S3150800F2F0A9F10104E31852F8044B43F8044B091F1B
S3150800F300F9D1ECE710BC704710B5074979441831B4
S3150800F310064C7C44163404E00A68081D11448847E4
S3150800F3200146A142F8D110BD2C0000004C00000097
S3150800F33005020602060307030803090309040A046B
S3150800F3400B040C040C050D050E050F050F0610061B
S3150800F350100710081DFFFFFFD01400001808002032
S3150800F3600000000079FFFFFF14000000680000009D
S3150800F370000000200000000000F00BF8002801D073
S3150800F380FFF7C2FF0020AFF30080FFF791FF00F000
S3150800F39002F80120704700F001B800000746384619
S3150800F3A000F002F8FBE7000080B5AFF30080024AE0
S3150800F3B011001820ABBEFBE726000200024885466E
S3150800F3C0024880470248004718080020A9F00008AC
S3150800F3D0E9F3000800000000010203040102030427
S3150800F3E006070809007A030AAFF30080AFF3008026
S3150800F3F0FFF7C2FFFFFFFFFFFFFF0000000000004E
S3150800F400FFFFFFFFFFF7FEBFFFF7FEBFFFF7FEBFD9
S3150800F410FFF7FEBFFFF7FEBFFFF7FEBFFFF7FEBF12
S3150800F420FFF7FEBFFFF7FEBFFFF7FEBFFFF7FEBF02
S3150800F430FFF7FEBFFFF7FEBFFFF7FEBFFFF7FEBFF2
S3150800F440FFF7FEBFFFF7FEBFFFF7FEBFFFF7FEBFE2
S3150800F450FFF7FEBFFFF7FEBFFFF7FEBFFFF7FEBFD2
S3150800F460FFF7FEBFFFF7FEBFFFF7FEBFFFF7FEBFC2
S3150800F470FFF7FEBFFFF7FEBFFFF7FEBFFFF7FEBFB2
S3150800F480FFF7FEBFFFF7FEBFFFF7FEBFFFF7FEBFA2
S3150800F490FFF7FEBFFFF7FEBFFFF7FEBFFFF7FEBF92
S3150800F4A0FFF7FEBFFFF7FEBFFFF7FEBFFFF7FEBF82
S3150800F4B0FFF7FEBFFFF7FEBFFFF7FEBFFFF7FEBF72
S3150800F4C0FFF7FEBFFFF7FEBFFFF7FEBFFFF7FEBF62
S3150800F4D0FFF7FEBFFFF7FEBFFFF7FEBFFFF7FEBF52
S3150800F4E0FFF7FEBFFFF7FEBFFFF7FEBFFFF7FEBF42
S3150800F4F0FFF7FEBFFFF7FEBFFFF7FEBFFFF7FEBF32
S3150800F500FFF7FEBFFFF7FEBFFFF7FEBFFFF7FEBF21
S3150800F510FFF7FEBFFFF7FEBFFFF7FEBFFFF7FEBF11
S3150800F520FFF7FEBFFFF7FEBFFFF7FEBFFFF7FEBF01
S3150800F530FFF7FEBFFFF7FEBFFFF7FEBFFFF7FEBFF1
S3150800F540FFF7FEBFFFF7FEBFFFF7FEBFFFF7FEBFE1
S3150800F550FFF7FEBFFFF7FEBFFFF7FEBFFFF7FEBFD1
S3110800F560FFF7FEBFFFF7FEBFFFF7FEBF78
S7050800F3E916
